:04000000B2017429AC
:100008000800A0002A0884002B1883172008800005
:10001800AA0A03146F29A9004030A0004B30A100A0
:100028004C30A400A5013A21AA012108031923286C
:100038002A145020FC3E031C2328AA145020200315
:10004800AB00280F2B28FF30A400A500362828086D
:10005800A500A401A600A7012B0A03193628A200AF
:10006800A3015421A90B4F281708CF39A41B203806
:10007800241B10380C389700250895008316861124
:1000880083122B088316920083121208FC392A0463
:10009800043892006F296F29A10CA00CA10CA00CA8
:1000A80008009818181218162C08A0002D08A1008E
:1000B800A201A3015F28602864008C1A7C28FF3005
:1000C800A207031CA307031CA007031CA107031C0A
:1000D8000800220F5E28230F5F28FA30A2000030A4
:1000E800A300602898181812181664008C1E792826
:1000F8001A0803146F290408A700851005100511B4
:1001080083168510051005110F3086058312270800
:10011800B218AB283A30A100FC3006213330A600D3
:10012800BF201030A10068300621BF2064300521AF
:100138002230A600BF202830AA200C30AA20013087
:10014800AA200630AA20B2142708AB283214A60029
:10015800321CB9280510033C031CBE28BE200730FA
:10016800A100D0300621031408003214FE3C031904
:100178006F290514321C321085140F3086052608A5
:10018800F03986048510A60E3218BF2832300521B2
:1001980003140800A400A90803196F2924086A2178
:1001A800A903D028A400290803196F292518831743
:1001B80024088400000883136A21A40AA903D82804
:1001C80083161C141A0883169B0A6F2903018316C9
:1001D8009A001C1555309D00AA309D009C149C184F
:1001E800F3281C119B0A6F29A301A200FF30A20764
:1001F800031CA307031C6F290330A100E630062166
:10020800FA28A101FC3EA000A109031C1129FF3016
:100218000000A00703180C29A0076400A10F0B29F0
:100228000800A101A301A20003302129A101A30113
:10023800A20006302129A2000530A80023082102C7
:10024800031D28292208200204300318013003194D
:1002580002302805031DFF306F290038031DFF30C9
:100268000405031DFF306F29A501A4011030A60065
:10027800210DA40DA50D2208A4022308031C230F99
:10028800A50203184E292208A40723080318230FE0
:10029800A5070310A00DA10DA60B3C2920086F2966
:1002A8001030A800A101A001A70CA60C031C62290C
:1002B8002208A00723080318230FA107A10CA00CEC
:1002C800A50CA40CA80B582924086F298400310810
:1002D8008A00300882008313031383126400080025
:1002E800831681309900203098008312903098004E
:1002F80007309F00C0308B008B1785298B1B0800A7
:10030800A42E822183168C1683128221E101822178
:10031800E201822183169B018312E42083160139AE
:1003280003191811031D1815831282218316013031
:100338009B008312E420831699008312822183167E
:1003480002309B008312E420D5008221DF01640083
:100358000E305F020318C729822104305F07D000DE
:1003680021300318013ED100500883169B008312E8
:10037800E420D000D1015F08383E84005008800096
:100388008221DF0FAB2982210130A300F430F9204C
:100398008221FE30802001308020FE3080200E3007
:1003A800802082215508A800FF30A2007F30A300DA
:1003B80001300F208221DE01822182216400831610
:1003C80083101819831483128318FA29822146305E
:1003D800AA00AB0139300520363005203030052021
:1003E800303005202030052082214B2A64008316F6
:1003F8008310181D8314831283184B2A82218221AB
:10040800640083161908403C8312031D1B2A8221AD
:100418004630AA00AB013130052039300520323092
:100428000520303005203030052082214A2A64001A
:1004380083161908203C8312031D322A8221463074
:10044800AA00AB01333005203830052034300520B0
:10045800303005203030052082214A2A6400831676
:100468001908153C8312031D492A82214630AA0027
:10047800AB013530052037300520363005203030C7
:1004880005203030052082214A2A822182218221BA
:10049800831603309B008312E420E4008221640069
:1004A8006408013C031D592AB023822164006108B5
:1004B80062020319AE2B8221E20A822164006208DB
:1004C800503C031D682AE20182216208A03E840094
:1004D8000008E000822164006008FE3C031DA72B91
:1004E8008221640061086202031D7C2A8221752A28
:1004F8008221E20A822164006208503C031D852A99
:10050800E20182216208A03E84000008CE00CF01EB
:1005180082218221A001A1014F08A3004E081F21BA
:10052800031D9A2A8221D4238221A52B0130A00001
:10053800A1014F08A3004E081F21031DA72A8221ED
:10054800DD238221A52B0230A000A1014F08A300C2
:100558004E081F21031DB42A8221E6238221A52BE0
:100568000330A000A1014F08A3004E081F21031D5E
:10057800C12A822108248221A52B0430A000A101D0
:100588004F08A3004E081F21031DCE2A82212A24CA
:100598008221A52B0530A000A1014F08A3004E0819
:1005A8001F21031DDB2A822131248221A52B06303D
:1005B800A000A1014F08A3004E081F21031DE82A2F
:1005C800822174248221A52B0730A000A1014F08A5
:1005D800A3004E081F21031DF52A82217F248221B2
:1005E800A52B0830A000A1014F08A3004E081F2129
:1005F800031D022B8221B0248221A52B0930A000E3
:10060800A1014F08A3004E081F21031D0F2B8221B3
:10061800BF248221A52B0A30A000A1014F08A30006
:100628004E081F21031D1C2B8221EB248221A52BA0
:100638000B30A000A1014F08A3004E081F21031D85
:10064800292B822105258221A52B0C30A000A10190
:100658004F08A3004E081F21031D442B8221831637
:1006680002309B0083125508EB208221E830AC0051
:100678000330AD005520031C592AE0008221A52B28
:100688000D30A000A1014F08A3004E081F21031D33
:10069800612B8221831602309B008312E420D5004F
:1006A80082215508A800FF30A2007F30A300013046
:1006B8000F208221592A8221A52B0E30A000A101EA
:1006C8004F08A3004E081F21031D6E2B82215E25B3
:1006D8008221A52B0F30A000A1014F08A3004E08CE
:1006E8001F21031D7B2B82218A258221A52B1030F7
:1006F800A000A1014F08A3004E081F21031D882B4D
:100708008221C4258221A52B1130A000A1014F0808
:10071800A3004E081F21031D952B8221FF2582214E
:10072800A52B1230A000A1014F08A3004E081F21DD
:10073800031DA22B82213A268221A52B8221592A28
:1007480082218221AD2B60088020DE0A7126652671
:10075800822182218221592A82210E30A9007F30EC
:10076800B000B101A5013830D6208221FE308020AA
:10077800C030802042308020613080207530802059
:10078800643080203A308020203080200530A90055
:100798007F30B000B101A5014630D6208221080083
:1007A8008221FE308020013080208221DE018221DA
:1007B80008008221FE308020023080208221DE0164
:1007C8008221080082217620E000822182216400B3
:1007D8006008003C031DF62B8221892682216526AC
:1007E8008221062C64006008013C031D032C822131
:1007F800DE0A82217126822165268221062C822129
:10080800592A82218221080082217620E000822153
:10081800822164006008003C031D182C82211830D6
:10082800CE00CF018221262C64006008013C031D04
:10083800232C82211C30CE00CF018221262C82213C
:100848000800822182215E268221080082217620EA
:10085800DE00822165268221080082217620E000C0
:100868008221822164006008003C031D412C822102
:100878000830CE00CF018221702C64006008013C52
:10088800031D4C2C82210C30CE00CF018221702C0C
:1008980064006008023C031D572C82210D30CE00F5
:1008A800CF018221702C64006008033C031D622C78
:1008B80082210E30CE00CF018221702C64006008A6
:1008C800043C031D6D2C82210F30CE00CF01822104
:1008D800702C82210800822182215E268221080054
:1008E800822189268221652682212030802082214A
:1008F80065268221080082217620D4007620D60041
:100908007620D7007620D8007620D9007620DA0025
:100918007620DB007620DC007620DD008221FE30A8
:10092800802040305407D000D101D10D50088020DC
:1009380056088020570880205808802059088020B1
:100948005A0880205B0880205C0880205D08802091
:10095800822165268221080082217620CE00CF01DF
:1009680082214E0880208221DE0A8221712682217E
:1009780065268221080082217620E00082218221DA
:1009880064006008003C031DD52C8221A801FF30BB
:10099800A2007F30A30001300F208221861182211E
:1009A800E92C64006008013C031DE62C8221A801A3
:1009B800FF30A2007F30A30001300F20822186156E
:1009C8008221E92C822108008221822108008221CB
:1009D8007620D50082216400013055020318F62CD8
:1009E8000130D5008221FA2CFF30D500822155082C
:1009F800A800FF30A2007F30A30001300F20822121
:100A0800080082217620E0008221822164006008AB
:100A1800003C031D1A2D822183161811831282218E
:100A2800831620309900831282214D2D64006008BE
:100A3800013C031D2A2D8221831618158312822159
:100A4800831640309900831282214D2D640060087E
:100A5800023C031D3A2D8221831618158312822128
:100A6800831620309900831282214D2D640060087E
:100A7800033C031D4A2D82218316181583128221F7
:100A8800831615309900831282214D2D822108008A
:100A98008221822183169B010030181901308312AC
:100AA800EB208221831601309B0019088312EB206A
:100AB8008221080082217620E300822182216400BD
:100AC8006308013C031D6D2D82218030E3008221E3
:100AD8007A2D64006308023C031D772D8221C03003
:100AE800E30082217A2D8221080082218221FE30B2
:100AF8008020630880201430A9007F30B000B10145
:100B08002030CE2082216526822108008221FF30F4
:100B1800D0005E08A0000F301A21D20050088400CF
:100B280052083121D200D30064005208530403193B
:100B3800A52D82214030DE00822165268221080011
:100B4800822182215E08A00040301521D0005E0875
:100B5800A0004F301A21D2005008840052083121D9
:100B6800D200D3006400520853040319C22D822115
:100B7800DE01822165268221080082218221080067
:100B88008221FF30D0005E08A0000F301A21D20069
:100B98005008840052083121D200D3006400520862
:100BA80053040319DF2D82214030DE078221652698
:100BB80082210800822182215E08A0004030152190
:100BC800D0005E08A0004F301A21D20050088400DF
:100BD80052083121D200D30064005208530403198B
:100BE800FD2D82214030DE02822165268221080007
:100BF8008221822108008221FF30D0005E08A000F7
:100C08000F301A21D2005008840052083121D20036
:100C1800D30064005208530403191A2E822140306D
:100C2800DE078221652682210800822182215E0852
:100C3800A00040301521D0005E08A0004F301A21D6
:100C4800D2005008840052083121D200D300640039
:100C5800520853040319382E82214030DE028221C3
:100C680065268221080082218221080082217620BF
:100C7800E0008221822164006008003C031D482EA8
:100C88008221E4018221552E64006008013C031D85
:100C9800522E82210130E4008221552E8221080043
:100CA80082218221831603309B0083126408EB2083
:100CB800822108008221FE3080204E088020822177
:100CC80008008221FE30802080305E07D000D101EC
:100CD800D10D5008802082210800822182216400E1
:100CE8005E08103C031D7D2E82214030DE008221EB
:100CF800872E64005E08503C031D862E8221DE018B
:100D08008221872E8221822108008221822164008B
:100D18005E08003C031D952E82214F30DE008221A3
:100D2800A22E64005E08403C031D9F2E82210F30D6
:100D3800DE008221A22E8221DE0382218221080088
:100D480064008C1EB62EE10A64006108503C031D45
:100D5800AE2EE1017620D000D1016108A03E8400CA
:060D6800500880000900A4
:02400E002E3F43
:1042000000002000FF0001004C004300440020009B
:1042100043006F006E00740072006F006C006C0051
:0442200065007200C3
:00000001FF
